 extevents001

 Timestamp is adf0e94a (reproducible build file hash)

 Preferred load address is 0000000180000000

 Start         Length     Name                   Class
 0001:00000000 00003a80H .text$mn                CODE
 0001:00003a80 00000036H .text$mn$00             CODE
 0001:00003ab6 00000092H .text$x                 CODE
 0002:00000000 000001d0H .idata$5                DATA
 0002:000001d0 00000038H .00cfg                  DATA
 0002:00000208 00000008H .CRT$XCA                DATA
 0002:00000210 00000008H .CRT$XCZ                DATA
 0002:00000218 00000008H .CRT$XIA                DATA
 0002:00000220 00000008H .CRT$XIC                DATA
 0002:00000228 00000008H .CRT$XIZ                DATA
 0002:00000230 00000008H .CRT$XLA                DATA
 0002:00000238 00000008H .CRT$XLZ                DATA
 0002:00000240 00000008H .CRT$XPA                DATA
 0002:00000248 00000008H .CRT$XPZ                DATA
 0002:00000250 00000008H .CRT$XTA                DATA
 0002:00000258 00000008H .CRT$XTZ                DATA
 0002:00000260 00000000H .gehcont$y              DATA
 0002:00000260 00000000H .gfids$y                DATA
 0002:00000260 000026a0H .rdata                  DATA
 0002:00002900 00000000H .rdata$CastGuardVftablesA DATA
 0002:00002900 00000000H .rdata$CastGuardVftablesC DATA
 0002:00002900 00000028H .rdata$T                DATA
 0002:00002928 000000bcH .rdata$voltmd           DATA
 0002:000029e4 0000031cH .rdata$zzzdbg           DATA
 0002:00002d00 00000008H .rtc$IAA                DATA
 0002:00002d08 00000008H .rtc$IZZ                DATA
 0002:00002d10 00000008H .rtc$TAA                DATA
 0002:00002d18 00000008H .rtc$TZZ                DATA
 0002:00002d20 00000004H .tls                    DATA
 0002:00002d24 00000004H .tls$                   DATA
 0002:00002d28 00000008H .tls$ZZZ                DATA
 0002:00002d30 00000350H .xdata                  DATA
 0002:00003080 00000364H .edata                  DATA
 0002:000033e4 0000008cH .idata$2                DATA
 0002:00003470 00000018H .idata$3                DATA
 0002:00003488 000001d0H .idata$4                DATA
 0002:00003658 00000490H .idata$6                DATA
 0003:00000000 00000080H .data                   DATA
 0003:00000080 0001b238H .bss                    DATA
 0004:00000000 000003ccH .pdata                  DATA

  Address         Publics by Value              Rva+Base               Lib:Object

 0000:00000000       __AbsoluteZero             0000000000000000     <absolute>
 0000:00000000       ___safe_se_handler_count   0000000000000000     <absolute>
 0000:00000000       ___safe_se_handler_table   0000000000000000     <absolute>
 0000:00000000       __arm64x_extra_rfe_table   0000000000000000     <absolute>
 0000:00000000       __arm64x_extra_rfe_table_size 0000000000000000     <absolute>
 0000:00000000       __arm64x_native_entrypoint 0000000000000000     <absolute>
 0000:00000000       __arm64x_redirection_metadata 0000000000000000     <absolute>
 0000:00000000       __arm64x_redirection_metadata_count 0000000000000000     <absolute>
 0000:00000000       __dynamic_value_reloc_table 0000000000000000     <absolute>
 0000:00000000       __enclave_config           0000000000000000     <absolute>
 0000:00000000       __guard_check_icall_a64n_fptr 0000000000000000     <absolute>
 0000:00000000       __guard_eh_cont_count      0000000000000000     <absolute>
 0000:00000000       __guard_eh_cont_table      0000000000000000     <absolute>
 0000:00000000       __guard_fids_count         0000000000000000     <absolute>
 0000:00000000       __guard_fids_table         0000000000000000     <absolute>
 0000:00000000       __guard_iat_count          0000000000000000     <absolute>
 0000:00000000       __guard_iat_table          0000000000000000     <absolute>
 0000:00000000       __guard_longjmp_count      0000000000000000     <absolute>
 0000:00000000       __guard_longjmp_table      0000000000000000     <absolute>
 0000:00000000       __hybrid_auxiliary_iat     0000000000000000     <absolute>
 0000:00000000       __hybrid_auxiliary_iat_copy 0000000000000000     <absolute>
 0000:00000000       __hybrid_code_map          0000000000000000     <absolute>
 0000:00000000       __hybrid_code_map_count    0000000000000000     <absolute>
 0000:00000000       __x64_code_ranges_to_entry_points 0000000000000000     <absolute>
 0000:00000000       __x64_code_ranges_to_entry_points_count 0000000000000000     <absolute>
 0000:00000100       __guard_flags              0000000000000100     <absolute>
 0000:00000000       __ImageBase                0000000180000000     <linker-defined>
 0001:00000000       ?NewObject@JNIEnv_@@QEAAPEAV_jobject@@PEAV_jclass@@PEAU_jmethodID@@ZZ 0000000180001000 f i libextevents001.obj
 0001:00000028       ?TranslateError@@YAPEBDW4jvmtiError@@@Z 0000000180001028 f   libextevents001.obj
 0001:000002e0       ?nsk_jni_check_exception@@YAHPEAUJNIEnv_@@QEBDH@Z 00000001800012e0 f   libextevents001.obj
 0001:00000424       ?nsk_jni_lverify@@YAHHPEAUJNIEnv_@@HQEBDH1ZZ 0000000180001424 f   libextevents001.obj
 0001:000004c4       Agent_Initialize           00000001800014c4 f   libextevents001.obj
 0001:00000654       Agent_OnAttach             0000000180001654 f   libextevents001.obj
 0001:00000654       Agent_OnLoad               0000000180001654 f   libextevents001.obj
 0001:0000065c       Java_nsk_jvmti_unit_FollowReferences_FollowRefObjects_addRefToVerify 000000018000165c f   libextevents001.obj
 0001:00000834       Java_nsk_jvmti_unit_FollowReferences_FollowRefObjects_getTag 0000000180001834 f   libextevents001.obj
 0001:000008f4       Java_nsk_jvmti_unit_FollowReferences_FollowRefObjects_resetRefsToVerify 00000001800018f4 f   libextevents001.obj
 0001:000008fc       Java_nsk_jvmti_unit_FollowReferences_FollowRefObjects_resetTags 00000001800018fc f   libextevents001.obj
 0001:00000940       Java_nsk_jvmti_unit_FollowReferences_FollowRefObjects_setTag 0000000180001940 f   libextevents001.obj
 0001:00000b98       Java_nsk_share_jvmti_ArgumentHandler_getAgentOptionsString 0000000180001b98 f   libextevents001.obj
 0001:00000c48       Java_nsk_share_jvmti_DebugeeClass_checkStatus 0000000180001c48 f   libextevents001.obj
 0001:00000cd0       Java_nsk_share_jvmti_DebugeeClass_resetAgentData 0000000180001cd0 f   libextevents001.obj
 0001:00000d30       Java_nsk_share_jvmti_RedefineAgent_agentStatus 0000000180001d30 f   libextevents001.obj
 0001:00000d3c       Java_nsk_share_jvmti_RedefineAgent_isRedefined 0000000180001d3c f   libextevents001.obj
 0001:00000d48       Java_nsk_share_jvmti_RedefineAgent_redefineAttempted 0000000180001d48 f   libextevents001.obj
 0001:00000d54       MA_checkStatus             0000000180001d54 f   libextevents001.obj
 0001:00000df8       __local_stdio_printf_options 0000000180001df8 f i libextevents001.obj
 0001:00001a30       exitOnError                0000000180002a30 f   libextevents001.obj
 0001:00001ae4       fprintf                    0000000180002ae4 f i libextevents001.obj
 0001:00001b28       nsk_complain               0000000180002b28 f   libextevents001.obj
 0001:00001b54       nsk_jvmti_createJVMTIEnv   0000000180002b54 f   libextevents001.obj
 0001:00001c84       nsk_jvmti_lverify          0000000180002c84 f   libextevents001.obj
 0001:00001d74       nsk_jvmti_parseOptions     0000000180002d74 f   libextevents001.obj
 0001:00001fc4       nsk_jvmti_resetAgentData   0000000180002fc4 f   libextevents001.obj
 0001:00002044       nsk_jvmti_resumeSync       0000000180003044 f   libextevents001.obj
 0001:000020ec       nsk_jvmti_setFailStatus    00000001800030ec f   libextevents001.obj
 0001:00002128       nsk_jvmti_waitForSync      0000000180003128 f   libextevents001.obj
 0001:0000222c       nsk_lcomplain              000000018000322c f   libextevents001.obj
 0001:0000224c       nsk_ldisplay               000000018000324c f   libextevents001.obj
 0001:0000226c       nsk_ltrace                 000000018000326c f   libextevents001.obj
 0001:0000228c       nsk_lvcomplain             000000018000328c f   libextevents001.obj
 0001:00002444       nsk_lvdisplay              0000000180003444 f   libextevents001.obj
 0001:00002490       nsk_lverify                0000000180003490 f   libextevents001.obj
 0001:000024ec       nsk_lvtrace                00000001800034ec f   libextevents001.obj
 0001:0000254c       nsk_printf                 000000018000354c f   libextevents001.obj
 0001:00002574       nsk_vprintf                0000000180003574 f   libextevents001.obj
 0001:00002628       printf                     0000000180003628 f i libextevents001.obj
 0001:00002b50       __raise_securityfailure    0000000180003b50 f   MSVCRT:gs_report.obj
 0001:00002b84       __report_gsfailure         0000000180003b84 f   MSVCRT:gs_report.obj
 0001:00002dc4       __GSHandlerCheck           0000000180003dc4 f   MSVCRT:gshandler.obj
 0001:00002de4       __GSHandlerCheckCommon     0000000180003de4 f   MSVCRT:gshandler.obj
 0001:00002e50       __security_check_cookie    0000000180003e50 f   MSVCRT:amdsecgs.obj
 0001:00003190       _DllMainCRTStartup         0000000180004190 f   MSVCRT:dll_dllmain.obj
 0001:000031d0       __scrt_acquire_startup_lock 00000001800041d0 f   MSVCRT:utility.obj
 0001:0000320c       __scrt_dllmain_after_initialize_c 000000018000420c f   MSVCRT:utility.obj
 0001:00003240       __scrt_dllmain_before_initialize_c 0000000180004240 f   MSVCRT:utility.obj
 0001:00003258       __scrt_dllmain_crt_thread_attach 0000000180004258 f   MSVCRT:utility.obj
 0001:00003280       __scrt_dllmain_crt_thread_detach 0000000180004280 f   MSVCRT:utility.obj
 0001:00003298       __scrt_dllmain_exception_filter 0000000180004298 f   MSVCRT:utility.obj
 0001:000032f8       __scrt_dllmain_uninitialize_c 00000001800042f8 f   MSVCRT:utility.obj
 0001:00003328       __scrt_dllmain_uninitialize_critical 0000000180004328 f   MSVCRT:utility.obj
 0001:0000333c       __scrt_initialize_crt      000000018000433c f   MSVCRT:utility.obj
 0001:00003388       __scrt_initialize_onexit_tables 0000000180004388 f   MSVCRT:utility.obj
 0001:00003414       __scrt_is_nonwritable_in_current_image 0000000180004414 f   MSVCRT:utility.obj
 0001:000034ac       __scrt_release_startup_lock 00000001800044ac f   MSVCRT:utility.obj
 0001:000034d0       __scrt_uninitialize_crt    00000001800044d0 f   MSVCRT:utility.obj
 0001:000034fc       _onexit                    00000001800044fc f   MSVCRT:utility.obj
 0001:00003538       atexit                     0000000180004538 f   MSVCRT:utility.obj
 0001:00003550       __crt_debugger_hook        0000000180004550 f   MSVCRT:utility_desktop.obj
 0001:00003558       __scrt_fastfail            0000000180004558 f   MSVCRT:utility_desktop.obj
 0001:000036a4       _guard_check_icall_nop     00000001800046a4 f i MSVCRT:guard_support.obj
 0001:000036a8       __security_init_cookie     00000001800046a8 f   MSVCRT:gs_support.obj
 0001:00003754       DllMain                    0000000180004754 f   MSVCRT:dll_dllmain_stub.obj
 0001:00003778       ?__scrt_initialize_type_info@@YAXXZ 0000000180004778 f   MSVCRT:tncleanup.obj
 0001:00003788       ?__scrt_uninitialize_type_info@@YAXXZ 0000000180004788 f   MSVCRT:tncleanup.obj
 0001:00003794       __local_stdio_scanf_options 0000000180004794 f i MSVCRT:default_local_stdio_options.obj
 0001:0000379c       __scrt_initialize_default_local_stdio_options 000000018000479c f   MSVCRT:default_local_stdio_options.obj
 0001:000037b8       __scrt_get_dyn_tls_init_callback 00000001800047b8 f   MSVCRT:dyn_tls_init.obj
 0001:000037c0       _RTC_Initialize            00000001800047c0 f   MSVCRT:initsect.obj
 0001:000037fc       _RTC_Terminate             00000001800047fc f   MSVCRT:initsect.obj
 0001:00003838       __isa_available_init       0000000180004838 f   MSVCRT:cpu_disp.obj
 0001:000039e4       _get_startup_argv_mode     00000001800049e4 f   MSVCRT:argv_mode.obj
 0001:000039ec       __scrt_is_ucrt_dll_in_use  00000001800049ec f   MSVCRT:ucrt_detection.obj
 0001:00003a00       memcpy                     0000000180004a00 f   vcruntime:VCRUNTIME140.dll
 0001:00003a06       memset                     0000000180004a06 f   vcruntime:VCRUNTIME140.dll
 0001:00003a0c       strchr                     0000000180004a0c f   vcruntime:VCRUNTIME140.dll
 0001:00003a12       strstr                     0000000180004a12 f   vcruntime:VCRUNTIME140.dll
 0001:00003a18       __C_specific_handler       0000000180004a18 f   vcruntime:VCRUNTIME140.dll
 0001:00003a1e       __std_type_info_destroy_list 0000000180004a1e f   vcruntime:VCRUNTIME140.dll
 0001:00003a24       strcmp                     0000000180004a24 f   ucrt:api-ms-win-crt-string-l1-1-0.dll
 0001:00003a2a       strlen                     0000000180004a2a f   ucrt:api-ms-win-crt-string-l1-1-0.dll
 0001:00003a30       _initterm                  0000000180004a30 f   ucrt:api-ms-win-crt-runtime-l1-1-0.dll
 0001:00003a36       _initterm_e                0000000180004a36 f   ucrt:api-ms-win-crt-runtime-l1-1-0.dll
 0001:00003a3c       _seh_filter_dll            0000000180004a3c f   ucrt:api-ms-win-crt-runtime-l1-1-0.dll
 0001:00003a42       _configure_narrow_argv     0000000180004a42 f   ucrt:api-ms-win-crt-runtime-l1-1-0.dll
 0001:00003a48       _initialize_narrow_environment 0000000180004a48 f   ucrt:api-ms-win-crt-runtime-l1-1-0.dll
 0001:00003a4e       _initialize_onexit_table   0000000180004a4e f   ucrt:api-ms-win-crt-runtime-l1-1-0.dll
 0001:00003a54       _register_onexit_function  0000000180004a54 f   ucrt:api-ms-win-crt-runtime-l1-1-0.dll
 0001:00003a5a       _execute_onexit_table      0000000180004a5a f   ucrt:api-ms-win-crt-runtime-l1-1-0.dll
 0001:00003a60       _crt_atexit                0000000180004a60 f   ucrt:api-ms-win-crt-runtime-l1-1-0.dll
 0001:00003a66       _cexit                     0000000180004a66 f   ucrt:api-ms-win-crt-runtime-l1-1-0.dll
 0001:00003a6c       __acrt_initialize          0000000180004a6c f   MSVCRT:ucrt_stubs.obj
 0001:00003a6c       __acrt_thread_attach       0000000180004a6c f   MSVCRT:ucrt_stubs.obj
 0001:00003a6c       __acrt_thread_detach       0000000180004a6c f   MSVCRT:ucrt_stubs.obj
 0001:00003a6c       __acrt_uninitialize        0000000180004a6c f   MSVCRT:ucrt_stubs.obj
 0001:00003a6c       __acrt_uninitialize_critical 0000000180004a6c f   MSVCRT:ucrt_stubs.obj
 0001:00003a6c       __scrt_stub_for_acrt_initialize 0000000180004a6c f   MSVCRT:ucrt_stubs.obj
 0001:00003a6c       __scrt_stub_for_acrt_thread_attach 0000000180004a6c f   MSVCRT:ucrt_stubs.obj
 0001:00003a6c       __scrt_stub_for_acrt_thread_detach 0000000180004a6c f   MSVCRT:ucrt_stubs.obj
 0001:00003a6c       __scrt_stub_for_acrt_uninitialize 0000000180004a6c f   MSVCRT:ucrt_stubs.obj
 0001:00003a6c       __scrt_stub_for_acrt_uninitialize_critical 0000000180004a6c f   MSVCRT:ucrt_stubs.obj
 0001:00003a6c       __vcrt_initialize          0000000180004a6c f   MSVCRT:ucrt_stubs.obj
 0001:00003a6c       __vcrt_thread_attach       0000000180004a6c f   MSVCRT:ucrt_stubs.obj
 0001:00003a6c       __vcrt_thread_detach       0000000180004a6c f   MSVCRT:ucrt_stubs.obj
 0001:00003a6c       __vcrt_uninitialize        0000000180004a6c f   MSVCRT:ucrt_stubs.obj
 0001:00003a6c       __vcrt_uninitialize_critical 0000000180004a6c f   MSVCRT:ucrt_stubs.obj
 0001:00003a70       __scrt_stub_for_is_c_termination_complete 0000000180004a70 f   MSVCRT:ucrt_stubs.obj
 0001:00003a70       _is_c_termination_complete 0000000180004a70 f   MSVCRT:ucrt_stubs.obj
 0001:00003a90       _guard_dispatch_icall_nop  0000000180004a90 f   MSVCRT:guard_dispatch.obj
 0001:00003ab0       _guard_xfg_dispatch_icall_nop 0000000180004ab0 f   MSVCRT:guard_xfg_dispatch.obj
 0002:00000000       __imp_RtlCaptureContext    0000000180005000     kernel32:KERNEL32.dll
 0002:00000008       __imp_RtlLookupFunctionEntry 0000000180005008     kernel32:KERNEL32.dll
 0002:00000010       __imp_RtlVirtualUnwind     0000000180005010     kernel32:KERNEL32.dll
 0002:00000018       __imp_UnhandledExceptionFilter 0000000180005018     kernel32:KERNEL32.dll
 0002:00000020       __imp_SetUnhandledExceptionFilter 0000000180005020     kernel32:KERNEL32.dll
 0002:00000028       __imp_GetCurrentProcess    0000000180005028     kernel32:KERNEL32.dll
 0002:00000030       __imp_TerminateProcess     0000000180005030     kernel32:KERNEL32.dll
 0002:00000038       __imp_IsProcessorFeaturePresent 0000000180005038     kernel32:KERNEL32.dll
 0002:00000040       __imp_CloseHandle          0000000180005040     kernel32:KERNEL32.dll
 0002:00000048       __imp_InitializeCriticalSectionAndSpinCount 0000000180005048     kernel32:KERNEL32.dll
 0002:00000050       __imp_DeleteCriticalSection 0000000180005050     kernel32:KERNEL32.dll
 0002:00000058       __imp_CreateEventW         0000000180005058     kernel32:KERNEL32.dll
 0002:00000060       __imp_GetModuleHandleW     0000000180005060     kernel32:KERNEL32.dll
 0002:00000068       __imp_GetProcAddress       0000000180005068     kernel32:KERNEL32.dll
 0002:00000070       __imp_IsDebuggerPresent    0000000180005070     kernel32:KERNEL32.dll
 0002:00000078       __imp_QueryPerformanceCounter 0000000180005078     kernel32:KERNEL32.dll
 0002:00000080       __imp_GetCurrentProcessId  0000000180005080     kernel32:KERNEL32.dll
 0002:00000088       __imp_GetCurrentThreadId   0000000180005088     kernel32:KERNEL32.dll
 0002:00000090       __imp_GetSystemTimeAsFileTime 0000000180005090     kernel32:KERNEL32.dll
 0002:00000098       __imp_DisableThreadLibraryCalls 0000000180005098     kernel32:KERNEL32.dll
 0002:000000a0       __imp_InitializeSListHead  00000001800050a0     kernel32:KERNEL32.dll
 0002:000000a8       \177KERNEL32_NULL_THUNK_DATA 00000001800050a8     kernel32:KERNEL32.dll
 0002:000000b0       __imp_memcpy               00000001800050b0     vcruntime:VCRUNTIME140.dll
 0002:000000b8       __imp_memset               00000001800050b8     vcruntime:VCRUNTIME140.dll
 0002:000000c0       __imp_strchr               00000001800050c0     vcruntime:VCRUNTIME140.dll
 0002:000000c8       __imp_strstr               00000001800050c8     vcruntime:VCRUNTIME140.dll
 0002:000000d0       __imp___C_specific_handler 00000001800050d0     vcruntime:VCRUNTIME140.dll
 0002:000000d8       __imp___std_type_info_destroy_list 00000001800050d8     vcruntime:VCRUNTIME140.dll
 0002:000000e0       \177VCRUNTIME140_NULL_THUNK_DATA 00000001800050e0     vcruntime:VCRUNTIME140.dll
 0002:000000e8       __imp_strtol               00000001800050e8     ucrt:api-ms-win-crt-convert-l1-1-0.dll
 0002:000000f0       \177api-ms-win-crt-convert-l1-1-0_NULL_THUNK_DATA 00000001800050f0     ucrt:api-ms-win-crt-convert-l1-1-0.dll
 0002:000000f8       __imp_malloc               00000001800050f8     ucrt:api-ms-win-crt-heap-l1-1-0.dll
 0002:00000100       __imp_free                 0000000180005100     ucrt:api-ms-win-crt-heap-l1-1-0.dll
 0002:00000108       \177api-ms-win-crt-heap-l1-1-0_NULL_THUNK_DATA 0000000180005108     ucrt:api-ms-win-crt-heap-l1-1-0.dll
 0002:00000110       __imp__errno               0000000180005110     ucrt:api-ms-win-crt-runtime-l1-1-0.dll
 0002:00000118       __imp_exit                 0000000180005118     ucrt:api-ms-win-crt-runtime-l1-1-0.dll
 0002:00000120       __imp__cexit               0000000180005120     ucrt:api-ms-win-crt-runtime-l1-1-0.dll
 0002:00000128       __imp__crt_atexit          0000000180005128     ucrt:api-ms-win-crt-runtime-l1-1-0.dll
 0002:00000130       __imp__execute_onexit_table 0000000180005130     ucrt:api-ms-win-crt-runtime-l1-1-0.dll
 0002:00000138       __imp__register_onexit_function 0000000180005138     ucrt:api-ms-win-crt-runtime-l1-1-0.dll
 0002:00000140       __imp__initialize_onexit_table 0000000180005140     ucrt:api-ms-win-crt-runtime-l1-1-0.dll
 0002:00000148       __imp__initialize_narrow_environment 0000000180005148     ucrt:api-ms-win-crt-runtime-l1-1-0.dll
 0002:00000150       __imp__configure_narrow_argv 0000000180005150     ucrt:api-ms-win-crt-runtime-l1-1-0.dll
 0002:00000158       __imp__seh_filter_dll      0000000180005158     ucrt:api-ms-win-crt-runtime-l1-1-0.dll
 0002:00000160       __imp__initterm_e          0000000180005160     ucrt:api-ms-win-crt-runtime-l1-1-0.dll
 0002:00000168       __imp__initterm            0000000180005168     ucrt:api-ms-win-crt-runtime-l1-1-0.dll
 0002:00000170       \177api-ms-win-crt-runtime-l1-1-0_NULL_THUNK_DATA 0000000180005170     ucrt:api-ms-win-crt-runtime-l1-1-0.dll
 0002:00000178       __imp___acrt_iob_func      0000000180005178     ucrt:api-ms-win-crt-stdio-l1-1-0.dll
 0002:00000180       __imp_fflush               0000000180005180     ucrt:api-ms-win-crt-stdio-l1-1-0.dll
 0002:00000188       __imp___stdio_common_vsprintf 0000000180005188     ucrt:api-ms-win-crt-stdio-l1-1-0.dll
 0002:00000190       __imp___stdio_common_vfprintf 0000000180005190     ucrt:api-ms-win-crt-stdio-l1-1-0.dll
 0002:00000198       \177api-ms-win-crt-stdio-l1-1-0_NULL_THUNK_DATA 0000000180005198     ucrt:api-ms-win-crt-stdio-l1-1-0.dll
 0002:000001a0       __imp_strcmp               00000001800051a0     ucrt:api-ms-win-crt-string-l1-1-0.dll
 0002:000001a8       __imp__strdup              00000001800051a8     ucrt:api-ms-win-crt-string-l1-1-0.dll
 0002:000001a8       __imp_strdup               00000001800051a8     ucrt:api-ms-win-crt-string-l1-1-0.dll
 0002:000001b0       __imp_strlen               00000001800051b0     ucrt:api-ms-win-crt-string-l1-1-0.dll
 0002:000001b8       __imp_strpbrk              00000001800051b8     ucrt:api-ms-win-crt-string-l1-1-0.dll
 0002:000001c0       __imp_strncpy              00000001800051c0     ucrt:api-ms-win-crt-string-l1-1-0.dll
 0002:000001c8       \177api-ms-win-crt-string-l1-1-0_NULL_THUNK_DATA 00000001800051c8     ucrt:api-ms-win-crt-string-l1-1-0.dll
 0002:000001d0       __guard_check_icall_fptr   00000001800051d0     MSVCRT:guard_support.obj
 0002:000001d8       __guard_xfg_check_icall_fptr 00000001800051d8     MSVCRT:guard_support.obj
 0002:000001e0       __guard_dispatch_icall_fptr 00000001800051e0     MSVCRT:guard_support.obj
 0002:000001e8       __guard_xfg_dispatch_icall_fptr 00000001800051e8     MSVCRT:guard_support.obj
 0002:000001f0       __guard_xfg_table_dispatch_icall_fptr 00000001800051f0     MSVCRT:guard_support.obj
 0002:000001f8       __castguard_check_failure_os_handled_fptr 00000001800051f8     MSVCRT:guard_support.obj
 0002:00000200       __guard_memcpy_fptr        0000000180005200     vcruntime:softmemtag.obj
 0002:00000208       __xc_a                     0000000180005208     MSVCRT:initializers.obj
 0002:00000210       __xc_z                     0000000180005210     MSVCRT:initializers.obj
 0002:00000218       __xi_a                     0000000180005218     MSVCRT:initializers.obj
 0002:00000228       __xi_z                     0000000180005228     MSVCRT:initializers.obj
 0002:00000230       __xl_a                     0000000180005230     MSVCRT:tlssup.obj
 0002:00000238       __xl_z                     0000000180005238     MSVCRT:tlssup.obj
 0002:00000240       __xp_a                     0000000180005240     MSVCRT:initializers.obj
 0002:00000248       __xp_z                     0000000180005248     MSVCRT:initializers.obj
 0002:00000250       __xt_a                     0000000180005250     MSVCRT:initializers.obj
 0002:00000258       __xt_z                     0000000180005258     MSVCRT:initializers.obj
 0002:00000260       g_refKindStr               0000000180005260     libextevents001.obj
 0002:00000410       ??_C@_09BPLDFGCI@unknown_0@ 0000000180005410     libextevents001.obj
 0002:00000420       ??_C@_0BL@FPNMECJD@JVMTI_HEAP_REFERENCE_CLASS@ 0000000180005420     libextevents001.obj
 0002:00000440       ??_C@_0BL@FKGKKLNM@JVMTI_HEAP_REFERENCE_FIELD@ 0000000180005440     libextevents001.obj
 0002:00000460       ??_C@_0CD@CAEHCFJF@JVMTI_HEAP_REFERENCE_ARRAY_ELEM@ 0000000180005460     libextevents001.obj
 0002:00000488       ??_C@_0CC@DNEBMCNK@JVMTI_HEAP_REFERENCE_CLASS_LOAD@ 0000000180005488     libextevents001.obj
 0002:000004b0       ??_C@_0BN@CJMIPEBB@JVMTI_HEAP_REFERENCE_SIGNERS@ 00000001800054b0     libextevents001.obj
 0002:000004d0       ??_C@_0CH@HBOIDPEB@JVMTI_HEAP_REFERENCE_PROTECTION@ 00000001800054d0     libextevents001.obj
 0002:000004f8       ??_C@_0BP@MDKGDGKL@JVMTI_HEAP_REFERENCE_INTERFACE@ 00000001800054f8     libextevents001.obj
 0002:00000518       ??_C@_0CC@JJMIHNJH@JVMTI_HEAP_REFERENCE_STATIC_FIE@ 0000000180005518     libextevents001.obj
 0002:00000540       ??_C@_0CD@IDHEEGID@JVMTI_HEAP_REFERENCE_CONSTANT_P@ 0000000180005540     libextevents001.obj
 0002:00000568       ??_C@_0CA@EFFCHNG@JVMTI_HEAP_REFERENCE_SUPERCLASS@ 0000000180005568     libextevents001.obj
 0002:00000588       ??_C@_0L@PCDFHGCJ@unknown_11@ 0000000180005588     libextevents001.obj
 0002:00000598       ??_C@_0L@NJBICFOK@unknown_12@ 0000000180005598     libextevents001.obj
 0002:000005a8       ??_C@_0L@MAADBEKL@unknown_13@ 00000001800055a8     libextevents001.obj
 0002:000005b8       ??_C@_0L@IPECICGM@unknown_14@ 00000001800055b8     libextevents001.obj
 0002:000005c8       ??_C@_0L@JGFJLDCN@unknown_15@ 00000001800055c8     libextevents001.obj
 0002:000005d8       ??_C@_0L@LNHEOAOO@unknown_16@ 00000001800055d8     libextevents001.obj
 0002:000005e8       ??_C@_0L@KEGPNBKP@unknown_17@ 00000001800055e8     libextevents001.obj
 0002:000005f8       ??_C@_0L@CDPHMNGA@unknown_18@ 00000001800055f8     libextevents001.obj
 0002:00000608       ??_C@_0L@DKOMPMCB@unknown_19@ 0000000180005608     libextevents001.obj
 0002:00000618       ??_C@_0L@OJGIPJDB@unknown_20@ 0000000180005618     libextevents001.obj
 0002:00000628       ??_C@_0CA@KAOFNDEM@JVMTI_HEAP_REFERENCE_JNI_GLOBAL@ 0000000180005628     libextevents001.obj
 0002:00000648       ??_C@_0CC@HPFAJBK@JVMTI_HEAP_REFERENCE_SYSTEM_CLA@ 0000000180005648     libextevents001.obj
 0002:00000670       ??_C@_0BN@FDEGFOHC@JVMTI_HEAP_REFERENCE_MONITOR@ 0000000180005670     libextevents001.obj
 0002:00000690       ??_C@_0CB@HKIBCMAJ@JVMTI_HEAP_REFERENCE_STACK_LOCA@ 0000000180005690     libextevents001.obj
 0002:000006b8       ??_C@_0BP@EAACMMOE@JVMTI_HEAP_REFERENCE_JNI_LOCAL@ 00000001800056b8     libextevents001.obj
 0002:000006d8       ??_C@_0BM@IJDEOGOE@JVMTI_HEAP_REFERENCE_THREAD@ 00000001800056d8     libextevents001.obj
 0002:000006f8       ??_C@_0BL@EDGPPKC@JVMTI_HEAP_REFERENCE_OTHER@ 00000001800056f8     libextevents001.obj
 0002:00000714       ??_C@_04BCJPDBDA@Code@     0000000180005714     libextevents001.obj
 0002:00000720       ??_C@_0BA@OCLMCFKC@LineNumberTable@ 0000000180005720     libextevents001.obj
 0002:00000730       ??_C@_0BD@CPAEPILC@LocalVariableTable@ 0000000180005730     libextevents001.obj
 0002:00000748       ??_C@_0BH@NMBDNHBD@LocalVariableTypeTable@ 0000000180005748     libextevents001.obj
 0002:00000760       ??_C@_0O@HIHEEDNJ@StackMapTable@ 0000000180005760     libextevents001.obj
 0002:00000770       ??_C@_0L@HCDIAMJG@?9?5?$CFs?0?5?$CFd?3?5@ 0000000180005770     libextevents001.obj
 0002:00000780       ??_C@_0JI@HLPECLFI@?$CD?5?4?4?4?6?$CD?5ERROR?3?5too?5many?5complai@ 0000000180005780     libextevents001.obj
 0002:00000820       ??_C@_0ED@JNEKCCOB@The?5following?5fake?5exception?5st@ 0000000180005820     libextevents001.obj
 0002:00000868       ??_C@_0CN@FCNMDFBH@nsk?4share?4Fake_Exception_for_RU@ 0000000180005868     libextevents001.obj
 0002:00000898       ??_C@_08PGFFNAEI@?$CI?$CFs?3?$CFd?$CJ?5@ 0000000180005898     libextevents001.obj
 0002:000008a8       ??_C@_0DP@IENMAEGI@s?2test?2hotspot?2jtreg?2vmTestbase@ 00000001800058a8     libextevents001.obj
 0002:000008e8       ??_C@_0BL@NDJLFFJB@?7at?5nsk_lvcomplain?$CI?$CFs?3?$CFd?$CJ?6@ 00000001800058e8     libextevents001.obj
 0002:00000908       ??_C@_0BC@JOOKAFKF@?$CD?5ERROR?3?5?$CFs?0?5?$CFd?3?5@ 0000000180005908     libextevents001.obj
 0002:00000920       ??_C@_09KJEAHMEH@?$CD?5ERROR?3?5@ 0000000180005920     libextevents001.obj
 0002:0000092c       ??_C@_02GPIOPFAK@?$DO?$DO@ 000000018000592c     libextevents001.obj
 0002:00000930       ??_C@_02FODMEDOG@?$DM?$DM@ 0000000180005930     libextevents001.obj
 0002:00000934       ??_C@_02DJGKEECL@?4?4@     0000000180005934     libextevents001.obj
 0002:00000938       ??_C@_0O@CJPGJOAF@?9?5?$CFs?0?5?$CFd?3?5?$CFs?5@ 0000000180005938     libextevents001.obj
 0002:00000948       ??_C@_0CB@IAKPDOIC@?$CD?5?5?5verified?5assertion?5is?5FALSE@ 0000000180005948     libextevents001.obj
 0002:00000970       ??_C@_0CO@LGONDEPD@stdout?3?5fflush?5failed?5?9?5err?$DN?$CFd?5@ 0000000180005970     libextevents001.obj
 0002:000009a0       ??_C@_0CO@KBGKJPBD@stderr?3?5fflush?5failed?5?9?5err?$DN?$CFd?5@ 00000001800059a0     libextevents001.obj
 0002:000009d0       ??_C@_06HPGEIPLA@?$DMnull?$DO@ 00000001800059d0     libextevents001.obj
 0002:000009d8       ??_C@_0BB@JCNMKLLK@JVMTI_ERROR_NONE@ 00000001800059d8     libextevents001.obj
 0002:000009f0       ??_C@_0BL@LDIMKLPH@JVMTI_ERROR_INVALID_THREAD@ 00000001800059f0     libextevents001.obj
 0002:00000a10       ??_C@_0CB@PJFPAIKJ@JVMTI_ERROR_INVALID_THREAD_GROU@ 0000000180005a10     libextevents001.obj
 0002:00000a38       ??_C@_0BN@LLMKHMNF@JVMTI_ERROR_INVALID_PRIORITY@ 0000000180005a38     libextevents001.obj
 0002:00000a58       ??_C@_0CB@MBOFKAGB@JVMTI_ERROR_THREAD_NOT_SUSPENDE@ 0000000180005a58     libextevents001.obj
 0002:00000a80       ??_C@_0BN@FABOLPBI@JVMTI_ERROR_THREAD_SUSPENDED@ 0000000180005a80     libextevents001.obj
 0002:00000aa0       ??_C@_0BN@FDGNOBJM@JVMTI_ERROR_THREAD_NOT_ALIVE@ 0000000180005aa0     libextevents001.obj
 0002:00000ac0       ??_C@_0BL@GOBIFKNJ@JVMTI_ERROR_INVALID_OBJECT@ 0000000180005ac0     libextevents001.obj
 0002:00000ae0       ??_C@_0BK@FCMAJPPC@JVMTI_ERROR_INVALID_CLASS@ 0000000180005ae0     libextevents001.obj
 0002:00000b00       ??_C@_0BP@IKLLBKEB@JVMTI_ERROR_CLASS_NOT_PREPARED@ 0000000180005b00     libextevents001.obj
 0002:00000b20       ??_C@_0BN@KLPPLKG@JVMTI_ERROR_INVALID_METHODID@ 0000000180005b20     libextevents001.obj
 0002:00000b40       ??_C@_0BN@BCEKOKND@JVMTI_ERROR_INVALID_LOCATION@ 0000000180005b40     libextevents001.obj
 0002:00000b60       ??_C@_0BM@DFDGPME@JVMTI_ERROR_INVALID_FIELDID@ 0000000180005b60     libextevents001.obj
 0002:00000b80       ??_C@_0BL@NELIEPEC@JVMTI_ERROR_NO_MORE_FRAMES@ 0000000180005b80     libextevents001.obj
 0002:00000ba0       ??_C@_0BJ@BDBECFDM@JVMTI_ERROR_OPAQUE_FRAME@ 0000000180005ba0     libextevents001.obj
 0002:00000bc0       ??_C@_0BK@MIIFNLOB@JVMTI_ERROR_TYPE_MISMATCH@ 0000000180005bc0     libextevents001.obj
 0002:00000be0       ??_C@_0BJ@HPCAOILC@JVMTI_ERROR_INVALID_SLOT@ 0000000180005be0     libextevents001.obj
 0002:00000c00       ??_C@_0BG@CHILOPNI@JVMTI_ERROR_DUPLICATE@ 0000000180005c00     libextevents001.obj
 0002:00000c18       ??_C@_0BG@DIEMLHKM@JVMTI_ERROR_NOT_FOUND@ 0000000180005c18     libextevents001.obj
 0002:00000c30       ??_C@_0BM@NHMCKHOB@JVMTI_ERROR_INVALID_MONITOR@ 0000000180005c30     libextevents001.obj
 0002:00000c50       ??_C@_0BO@PPEDAJGL@JVMTI_ERROR_NOT_MONITOR_OWNER@ 0000000180005c50     libextevents001.obj
 0002:00000c70       ??_C@_0BG@FCAIPEID@JVMTI_ERROR_INTERRUPT@ 0000000180005c70     libextevents001.obj
 0002:00000c88       ??_C@_0CB@EGDBNKOI@JVMTI_ERROR_INVALID_CLASS_FORMA@ 0000000180005c88     libextevents001.obj
 0002:00000cb0       ??_C@_0CG@DGKOGIAL@JVMTI_ERROR_CIRCULAR_CLASS_DEFI@ 0000000180005cb0     libextevents001.obj
 0002:00000cd8       ??_C@_0BP@ICEALPKC@JVMTI_ERROR_FAILS_VERIFICATION@ 0000000180005cd8     libextevents001.obj
 0002:00000cf8       ??_C@_0DC@JDACLMIO@JVMTI_ERROR_UNSUPPORTED_REDEFIN@ 0000000180005cf8     libextevents001.obj
 0002:00000d30       ??_C@_0DE@GKDKNOMJ@JVMTI_ERROR_UNSUPPORTED_REDEFIN@ 0000000180005d30     libextevents001.obj
 0002:00000d68       ??_C@_0BO@LAFKIOG@JVMTI_ERROR_INVALID_TYPESTATE@ 0000000180005d68     libextevents001.obj
 0002:00000d88       ??_C@_0DH@INDGCLLB@JVMTI_ERROR_UNSUPPORTED_REDEFIN@ 0000000180005d88     libextevents001.obj
 0002:00000dc0       ??_C@_0DE@NHEOMMGI@JVMTI_ERROR_UNSUPPORTED_REDEFIN@ 0000000180005dc0     libextevents001.obj
 0002:00000df8       ??_C@_0CA@EKPNJOEP@JVMTI_ERROR_UNSUPPORTED_VERSION@ 0000000180005df8     libextevents001.obj
 0002:00000e18       ??_C@_0BN@OFFMAHHL@JVMTI_ERROR_NAMES_DONT_MATCH@ 0000000180005e18     libextevents001.obj
 0002:00000e38       ??_C@_0DN@HHBBLAKE@JVMTI_ERROR_UNSUPPORTED_REDEFIN@ 0000000180005e38     libextevents001.obj
 0002:00000e78       ??_C@_0DO@HMBGBGNA@JVMTI_ERROR_UNSUPPORTED_REDEFIN@ 0000000180005e78     libextevents001.obj
 0002:00000eb8       ??_C@_0BP@PBECGKHJ@JVMTI_ERROR_UNMODIFIABLE_CLASS@ 0000000180005eb8     libextevents001.obj
 0002:00000ed8       ??_C@_0BK@CANILEHF@JVMTI_ERROR_NOT_AVAILABLE@ 0000000180005ed8     libextevents001.obj
 0002:00000ef8       ??_C@_0CE@INJKMEFK@JVMTI_ERROR_MUST_POSSESS_CAPABI@ 0000000180005ef8     libextevents001.obj
 0002:00000f20       ??_C@_0BJ@LBFPFPDM@JVMTI_ERROR_NULL_POINTER@ 0000000180005f20     libextevents001.obj
 0002:00000f40       ??_C@_0BP@CHJPNNEM@JVMTI_ERROR_ABSENT_INFORMATION@ 0000000180005f40     libextevents001.obj
 0002:00000f60       ??_C@_0BP@OMFMNLC@JVMTI_ERROR_INVALID_EVENT_TYPE@ 0000000180005f60     libextevents001.obj
 0002:00000f80       ??_C@_0BN@BIBNPHHO@JVMTI_ERROR_ILLEGAL_ARGUMENT@ 0000000180005f80     libextevents001.obj
 0002:00000fa0       ??_C@_0BK@KKNDHDCE@JVMTI_ERROR_NATIVE_METHOD@ 0000000180005fa0     libextevents001.obj
 0002:00000fc0       ??_C@_0BK@PMKCFHAE@JVMTI_ERROR_OUT_OF_MEMORY@ 0000000180005fc0     libextevents001.obj
 0002:00000fe0       ??_C@_0BK@NNJBDMNB@JVMTI_ERROR_ACCESS_DENIED@ 0000000180005fe0     libextevents001.obj
 0002:00001000       ??_C@_0BI@GHECLMNC@JVMTI_ERROR_WRONG_PHASE@ 0000000180006000     libextevents001.obj
 0002:00001018       ??_C@_0BF@OLIHJOII@JVMTI_ERROR_INTERNAL@ 0000000180006018     libextevents001.obj
 0002:00001030       ??_C@_0BO@EOHGKJHI@JVMTI_ERROR_UNATTACHED_THREAD@ 0000000180006030     libextevents001.obj
 0002:00001050       ??_C@_0CA@LKHFDACL@JVMTI_ERROR_INVALID_ENVIRONMENT@ 0000000180006050     libextevents001.obj
 0002:00001070       ??_C@_0BA@MMFHLOKK@?$DMunknown?5error?$DO@ 0000000180006070     libextevents001.obj
 0002:00001080       ??_C@_0CF@CBHOKDB@throwable?5?$DN?5jni?9?$DOExceptionOccur@ 0000000180006080     libextevents001.obj
 0002:000010a8       ??_C@_03OFAPEBGM@?$CFs?6@  00000001800060a8     libextevents001.obj
 0002:000010b0       ??_C@_0DM@LPIGEGNJ@s?2test?2hotspot?2jtreg?2vmTestbase@ 00000001800060b0     libextevents001.obj
 0002:000010f0       ??_C@_0CC@NFCNPEPK@Exception?5in?5JNI?5call?5?$CIcleared?$CJ@ 00000001800060f0     libextevents001.obj
 0002:00001118       ??_C@_0BJ@IBAKFIKF@jni?9?$DOExceptionDescribe?$CI?$CJ@ 0000000180006118     libextevents001.obj
 0002:00001138       ??_C@_0BG@GGKALKMH@jni?9?$DOExceptionClear?$CI?$CJ@ 0000000180006138     libextevents001.obj
 0002:00001150       ??_C@_0CF@JMGFGJLJ@?$CD?5?5?5verified?5JNI?5assertion?5is?5F@ 0000000180006150     libextevents001.obj
 0002:00001178       ??_C@_07KBAMPNJK@verbose@  0000000180006178     libextevents001.obj
 0002:00001180       ??_C@_0DN@PKJBOLAP@nsk_jvmti_parseOptions?$CI?$CJ?3?5unexp@ 0000000180006180     libextevents001.obj
 0002:000011c0       ??_C@_05IMBNNINJ@trace@    00000001800061c0     libextevents001.obj
 0002:000011c8       ??_C@_0DD@BJKGNDMB@nsk_jvmti_parseOptions?$CI?$CJ?3?5no?5va@ 00000001800061c8     libextevents001.obj
 0002:000011fc       ??_C@_04CGFJFPFD@none@     00000001800061fc     libextevents001.obj
 0002:00001204       ??_C@_06BMELKFMA@before@   0000000180006204     libextevents001.obj
 0002:0000120c       ??_C@_05CMKPCFDK@after@    000000018000620c     libextevents001.obj
 0002:00001214       ??_C@_03NFKEKGGK@all@      0000000180006214     libextevents001.obj
 0002:00001218       ??_C@_0DM@NDNJGJKE@nsk_jvmti_parseOptions?$CI?$CJ?3?5uexpe@ 0000000180006218     libextevents001.obj
 0002:00001258       ??_C@_08NBBJKJO@waittime@  0000000180006258     libextevents001.obj
 0002:00001268       ??_C@_0DO@CMHGAOHC@nsk_jvmti_parseOptions?$CI?$CJ?3?5not?5i@ 0000000180006268     libextevents001.obj
 0002:000012a8       ??_C@_0DL@LNMPBDLN@nsk_jvmti_parseOptions?$CI?$CJ?3?5negat@ 00000001800062a8     libextevents001.obj
 0002:000012e8       ??_C@_0DA@GMFJNOJH@nsk_jvmti_parseOptions?$CI?$CJ?3?5unkno@ 00000001800062e8     libextevents001.obj
 0002:00001318       ??_C@_0CO@CCIAMEAN@nsk_jvmti_parseOptions?$CI?$CJ?3?5found@ 0000000180006318     libextevents001.obj
 0002:00001348       ??_C@_0CJ@OEGPCGDL@nsk_jvmti_parseOptions?$CI?$CJ?3?5out?5o@ 0000000180006348     libextevents001.obj
 0002:00001378       ??_C@_0DI@NMBHPGGF@nsk_jvmti_parseOptions?$CI?$CJ?3?5too?5m@ 0000000180006378     libextevents001.obj
 0002:000013b0       ??_C@_03POGCGECB@?5?0?$HO@ 00000001800063b0     libextevents001.obj
 0002:000013b8       ??_C@_0CB@MLNJNCLJ@?5?5jvmti?5error?3?5code?$DN?$CFd?0?5name?$DN?$CFs@ 00000001800063b8     libextevents001.obj
 0002:000013e0       ??_C@_0CD@OHBGDKMK@?$CD?5?5?5jvmti?5error?3?5code?$DN?$CFd?0?5name?$DN@ 00000001800063e0     libextevents001.obj
 0002:00001408       ??_C@_0CG@JNNCGPHB@?$CD?5?5?5error?5expected?3?5code?$DN?$CFd?0?5na@ 0000000180006408     libextevents001.obj
 0002:00001430       ??_C@_0EB@IMGKPCGE@?$CIstr_obj?5?$DN?5jni?9?$DONewStringUTF?$CIco@ 0000000180006430     libextevents001.obj
 0002:00001480       ??_C@_0EA@HFOGGBCC@s?2test?2hotspot?2jtreg?2vmTestbase@ 0000000180006480     libextevents001.obj
 0002:000014c0       ??_C@_05KKCIMGE@error@     00000001800064c0     libextevents001.obj
 0002:000014c8       ??_C@_0CJ@JACLEAA@Test?5failed?5by?5setFailStatus?$CI?$CJ?4@ 00000001800064c8     libextevents001.obj
 0002:000014f8       ??_C@_0BD@HGNAOMCP@agent_data_monitor@ 00000001800064f8     libextevents001.obj
 0002:00001510       ??_C@_0EB@OGCLGKLN@javaVM?9?$DOGetEnv?$CI?$CIvoid?5?$CK?$CK?$CJ?$CGjvmti_@ 0000000180006510     libextevents001.obj
 0002:00001560       ??_C@_0EA@PNBCDMOA@s?2test?2hotspot?2jtreg?2vmTestbase@ 0000000180006560     libextevents001.obj
 0002:000015a0       ??_C@_0CI@DDPIFBGM@init_agent_data?$CIjvmti_env?0?5?$CGage@ 00000001800065a0     libextevents001.obj
 0002:000015c8       ??_C@_0DI@ILAHDLMP@?$CI?$CKagentThreadProc?$CJ?$CIjvmti_env?0?5a@ 00000001800065c8     libextevents001.obj
 0002:00001600       ??_C@_0BD@KDBALNLB@JVMTI?5agent?5thread@ 0000000180006600     libextevents001.obj
 0002:00001618       ??_C@_0BB@NOKBFPFO@java?1lang?1Thread@ 0000000180006618     libextevents001.obj
 0002:0000162c       ??_C@_06FALKBLGB@?$DMinit?$DO@ 000000018000662c     libextevents001.obj
 0002:00001638       ??_C@_0BG@IKDDPPGD@?$CILjava?1lang?1String?$DL?$CJV@ 0000000180006638     libextevents001.obj
 0002:00001650       ??_C@_0EB@IFJBFEKC@?$CIthreadClass?5?$DN?5jni_env?9?$DOFindCla@ 0000000180006650     libextevents001.obj
 0002:000016a0       ??_C@_0GF@FGFIBKKL@?$CIthreadCtor?5?$DN?5jni_env?9?$DOGetMetho@ 00000001800066a0     libextevents001.obj
 0002:00001708       ??_C@_0DN@NCPDJLOG@?$CIthreadName?5?$DN?5jni_env?9?$DONewStrin@ 0000000180006708     libextevents001.obj
 0002:00001750       ??_C@_0FE@PFKODBGC@?$CIthreadObject?5?$DN?5jni_env?9?$DONewObj@ 0000000180006750     libextevents001.obj
 0002:000017b0       ??_C@_0ED@HOBAHHJI@?$CIthreadGlobalRef?5?$DN?5jni_env?9?$DONew@ 00000001800067b0     libextevents001.obj
 0002:00001800       ??_C@_0FN@HNJJAHFC@jvmti_env?9?$DORunAgentThread?$CIagent@ 0000000180006800     libextevents001.obj
 0002:00001860       ??_C@_0EA@MOJDNKDF@Debuggee?5status?5sync?5aborted?5be@ 0000000180006860     libextevents001.obj
 0002:000018a0       ??_C@_0CO@PGPGMHBJ@No?5status?5sync?5occured?5for?5time@ 00000001800068a0     libextevents001.obj
 0002:000018d0       ??_C@_0CL@DOEBDPKJ@Debuggee?5was?5not?5suspended?5on?5s@ 00000001800068d0     libextevents001.obj
 0002:00001900       ??_C@_0EA@EEOEJAEN@status?5?$DN?5syncDebuggeeStatus?$CIjni@ 0000000180006900     libextevents001.obj
 0002:00001940       ??_C@_0BL@JBCFNBMB@nsk_jvmti_resetAgentData?$CI?$CJ@ 0000000180006940     libextevents001.obj
 0002:00001960       ??_C@_0EL@LPBEELIP@s?2test?2hotspot?2jtreg?2vmTestbase@ 0000000180006960     libextevents001.obj
 0002:000019b0       ??_C@_0CK@JDAMFDMJ@jvmti?9?$DOSetTag?$CIo?0?5tag?$CJ?5?$DN?$DN?5JVMTI_@ 00000001800069b0     libextevents001.obj
 0002:000019e0       ??_C@_0CC@DAMNHKNI@Can?8t?5set?5tag?5?$CFli?5for?5object?5?$CFl@ 00000001800069e0     libextevents001.obj
 0002:00001a08       ??_C@_0DL@HAJPNKEF@jvmti?9?$DOGetObjectHashCode?$CIo?0?5?$CGha@ 0000000180006a08     libextevents001.obj
 0002:00001a48       ??_C@_0BL@JFPIEOBF@Can?8t?5get?5hash?5object?5?$CFlx?6@ 0000000180006a48     libextevents001.obj
 0002:00001a68       ??_C@_0BG@DICPHBKN@setTag?3?5?$CF08x?5?$DM?9?5?$CF?53li@ 0000000180006a68     libextevents001.obj
 0002:00001a80       ??_C@_0DH@FCEEBDMJ@?$CIs?5?$DN?5jni?9?$DOGetStringUTFChars?$CIsIn@ 0000000180006a80     libextevents001.obj
 0002:00001ab8       ??_C@_0BJ@OKKGHDCN@Can?8t?5get?5string?5at?5?$CF?$CDp?6@ 0000000180006ab8     libextevents001.obj
 0002:00001ad8       ??_C@_0BP@EKFLGGFJ@Can?8t?5get?5string?5at?5?$CF?$CDp?3?5null?6@ 0000000180006ad8     libextevents001.obj
 0002:00001af8       ??_C@_06ICODBHCL@?5?1?1?5?$CFs@ 0000000180006af8     libextevents001.obj
 0002:00001b00       ??_C@_0DB@KGFPLEGO@?$CIr?5?$DN?5jvmti?9?$DOGetTag?$CIo?0?5?$CGtag?$CJ?$CJ?5?$DN?$DN@ 0000000180006b00     libextevents001.obj
 0002:00001b38       ??_C@_0CO@PDAGBCGJ@Can?8t?5GetTag?5for?5object?5?$CFlx?4?5Re@ 0000000180006b38     libextevents001.obj
 0002:00001b68       ??_C@_0CH@HPEODOHC@TEST_BUG?3?5Max?4?5number?5of?5refs?5r@ 0000000180006b68     libextevents001.obj
 0002:00001b90       ??_C@_0DI@PHFCABIM@?$CIr?5?$DN?5jvmti?9?$DOGetTag?$CIfrom?0?5?$CGtagFr@ 0000000180006b90     libextevents001.obj
 0002:00001bc8       ??_C@_0DI@MDEGFNKD@TEST_BUG?3?5Can?8t?5GetTag?5for?5obje@ 0000000180006bc8     libextevents001.obj
 0002:00001c00       ??_C@_0DE@MLELJAHM@?$CIr?5?$DN?5jvmti?9?$DOGetTag?$CIto?0?5?$CGtagTo?$CJ?$CJ@ 0000000180006c00     libextevents001.obj
 0002:00001c38       ??_C@_0BL@ODLJGGAH@Get?5extension?5events?5list?6@ 0000000180006c38     libextevents001.obj
 0002:00001c60       ??_C@_0FL@ODFKIINH@s?2test?2hotspot?2jtreg?2vmTestbase@ 0000000180006c60     libextevents001.obj
 0002:00001cc0       ??_C@_0CP@LJBAKDOL@jvmti?9?$DOGetExtensionEvents?$CI?$CGextC@ 0000000180006cc0     libextevents001.obj
 0002:00001cf0       ??_C@_0BF@BELKDIBL@?5?5?4?4?4?5got?5count?3?5?$CFd?6@ 0000000180006cf0     libextevents001.obj
 0002:00001d08       ??_C@_0BH@MKCPOPGG@?5?5?4?4?4?5got?5list?3?5?50x?$CFp?6@ 0000000180006d08     libextevents001.obj
 0002:00001d20       ??_C@_0HB@IJGCOLIE@In?5?$CFs?5phase?5GetExtensionEvents?$CI@ 0000000180006d20     libextevents001.obj
 0002:00001d98       ??_C@_0CI@HOFOGCCH@Check?5each?5extension?5events?3?5?$CFd@ 0000000180006d98     libextevents001.obj
 0002:00001dc0       ??_C@_0O@FNLODKDN@?5?5event?5?$CD?$CFd?3?6@ 0000000180006dc0     libextevents001.obj
 0002:00001dd0       ??_C@_0BF@KFKFLBKC@?5?5?5?5event_index?3?5?$CFd?6@ 0000000180006dd0     libextevents001.obj
 0002:00001de8       ??_C@_0BH@KHKANFDN@?5?5?5?5id?3?5?5?5?5?5?5?5?5?5?5?$CC?$CFs?$CC?6@ 0000000180006de8     libextevents001.obj
 0002:00001e00       ??_C@_0BH@OEJLADBN@?5?5?5?5short_desc?3?5?5?$CC?$CFs?$CC?6@ 0000000180006e00     libextevents001.obj
 0002:00001e18       ??_C@_0BF@MLPNJJID@?5?5?5?5param_count?3?5?$CFd?6@ 0000000180006e18     libextevents001.obj
 0002:00001e30       ??_C@_0BH@FJBPHKIN@?5?5?5?5params?3?5?5?5?5?5?50x?$CFp?6@ 0000000180006e30     libextevents001.obj
 0002:00001e48       ??_C@_0BC@GNEIHHHK@?5?5?5?5?5?5param?5?$CD?$CFd?3?6@ 0000000180006e48     libextevents001.obj
 0002:00001e60       ??_C@_0BJ@JEOHHFPP@?5?5?5?5?5?5?5?5name?3?5?5?5?5?5?5?$CC?$CFs?$CC?6@ 0000000180006e60     libextevents001.obj
 0002:00001e80       ??_C@_0BH@HMFNJCBE@?5?5?5?5?5?5?5?5kind?3?5?5?5?5?5?5?$CFd?6@ 0000000180006e80     libextevents001.obj
 0002:00001e98       ??_C@_0BH@PPCNHCAG@?5?5?5?5?5?5?5?5base_type?3?5?$CFd?6@ 0000000180006e98     libextevents001.obj
 0002:00001eb0       ??_C@_0BH@JKEDJEAF@?5?5?5?5?5?5?5?5null_ok?3?5?5?5?$CFd?6@ 0000000180006eb0     libextevents001.obj
 0002:00001ed0       ??_C@_0MB@JGIHKLDE@In?5?$CFs?5phase?5GetExtensionEvents?$CI@ 0000000180006ed0     libextevents001.obj
 0002:00001fa0       ??_C@_0JI@MFLFKFCO@In?5?$CFs?5phase?5GetExtensionEvents?$CI@ 0000000180006fa0     libextevents001.obj
 0002:00002038       ??_C@_0BA@NKOLBGI@com?4sun?4hotspot@ 0000000180007038     libextevents001.obj
 0002:00002050       ??_C@_0JN@CPJCBPJD@In?5?$CFs?5phase?5GetExtensionEvents?$CI@ 0000000180007050     libextevents001.obj
 0002:000020f0       ??_C@_0JK@CLKFNFBK@In?5?$CFs?5phase?5GetExtensionEvents?$CI@ 00000001800070f0     libextevents001.obj
 0002:00002190       ??_C@_0MH@OPOIIMGE@In?5?$CFs?5phase?5GetExtensionEvents?$CI@ 0000000180007190     libextevents001.obj
 0002:00002260       ??_C@_0NF@MKNJIBGH@In?5?$CFs?5phase?5GetExtensionEvents?$CI@ 0000000180007260     libextevents001.obj
 0002:00002340       ??_C@_0NF@CHDHHBKP@In?5?$CFs?5phase?5GetExtensionEvents?$CI@ 0000000180007340     libextevents001.obj
 0002:00002418       ??_C@_0CI@EPFKJIGD@Deallocate?5extension?5events?5lis@ 0000000180007418     libextevents001.obj
 0002:00002440       ??_C@_0CL@KGKEDHBN@jvmti?9?$DODeallocate?$CI?$CIunsigned?5cha@ 0000000180007440     libextevents001.obj
 0002:00002470       ??_C@_0BD@PFBGGHID@?5?5?4?4?4?5deallocated?6@ 0000000180007470     libextevents001.obj
 0002:00002488       ??_C@_0BO@HLANDLHM@Wait?5for?5debugee?5class?5ready?6@ 0000000180007488     libextevents001.obj
 0002:000024a8       ??_C@_0BP@LAIJOMPC@nsk_jvmti_waitForSync?$CItimeout?$CJ@ 00000001800074a8     libextevents001.obj
 0002:000024c8       ??_C@_0DH@FMCJOOIC@?$DO?$DO?$DO?5Testcase?5?$CD2?3?5Check?5extensio@ 00000001800074c8     libextevents001.obj
 0002:00002500       ??_C@_04GLMHKBCH@live@     0000000180007500     libextevents001.obj
 0002:00002508       ??_C@_0BH@HPEOJMHL@Let?5debugee?5to?5finish?6@ 0000000180007508     libextevents001.obj
 0002:00002520       ??_C@_0BH@LECMGIIA@nsk_jvmti_resumeSync?$CI?$CJ@ 0000000180007520     libextevents001.obj
 0002:00002538       ??_C@_0CA@MNKGCBCG@nsk_jvmti_parseOptions?$CIoptions?$CJ@ 0000000180007538     libextevents001.obj
 0002:00002558       ??_C@_0DN@MIAMNFPH@?$CIjvmti?5?$DN?5nsk_jvmti_createJVMTIE@ 0000000180007558     libextevents001.obj
 0002:00002598       ??_C@_0DJ@NCCEMECG@?$DO?$DO?$DO?5Testcase?5?$CD1?3?5Check?5extensio@ 0000000180007598     libextevents001.obj
 0002:000025d4       ??_C@_06FEOMBGJC@OnLoad@   00000001800075d4     libextevents001.obj
 0002:000025e0       ??_C@_0CL@PIACJIPK@nsk_jvmti_setAgentProc?$CIagentPro@ 00000001800075e0     libextevents001.obj
 0002:00002620       ??_C@_1EC@JIJBPKFM@?$AAa?$AAp?$AAi?$AA?9?$AAm?$AAs?$AA?9?$AAw?$AAi?$AAn?$AA?9?$AAc?$AAo?$AAr?$AAe@ 0000000180007620     MSVCRT:thread_safe_statics.obj
 0002:00002668       ??_C@_1BK@MGMFAEKH@?$AAk?$AAe?$AAr?$AAn?$AAe?$AAl?$AA3?$AA2?$AA?4?$AAd?$AAl?$AAl@ 0000000180007668     MSVCRT:thread_safe_statics.obj
 0002:00002688       ??_C@_0BJ@JEBJOJFJ@SleepConditionVariableCS@ 0000000180007688     MSVCRT:thread_safe_statics.obj
 0002:000026a8       ??_C@_0BJ@PGPPEPCC@WakeAllConditionVariable@ 00000001800076a8     MSVCRT:thread_safe_statics.obj
 0002:000026c8       _pDefaultRawDllMain        00000001800076c8     MSVCRT:dll_dllmain.obj
 0002:000026c8       _pRawDllMain               00000001800076c8     MSVCRT:dll_dllmain.obj
 0002:000026d0       __xmm@ffffffffffffffffffffffffffffffff 00000001800076d0     MSVCRT:utility.obj
 0002:000026e0       _load_config_used          00000001800076e0     MSVCRT:loadcfg.obj
 0002:00002900       _tls_used                  0000000180007900     MSVCRT:tlssup.obj
 0002:00002928       __volatile_metadata        0000000180007928     <linker-defined>
 0002:00002d00       __rtc_iaa                  0000000180007d00     MSVCRT:initsect.obj
 0002:00002d08       __rtc_izz                  0000000180007d08     MSVCRT:initsect.obj
 0002:00002d10       __rtc_taa                  0000000180007d10     MSVCRT:initsect.obj
 0002:00002d18       __rtc_tzz                  0000000180007d18     MSVCRT:initsect.obj
 0002:00002d20       _tls_start                 0000000180007d20     MSVCRT:tlssup.obj
 0002:00002d24       _Init_thread_epoch         0000000180007d24     MSVCRT:thread_safe_statics.obj
 0002:00002d28       _tls_end                   0000000180007d28     MSVCRT:tlssup.obj
 0002:000033e4       __IMPORT_DESCRIPTOR_KERNEL32 00000001800083e4     kernel32:KERNEL32.dll
 0002:000033f8       __IMPORT_DESCRIPTOR_VCRUNTIME140 00000001800083f8     vcruntime:VCRUNTIME140.dll
 0002:0000340c       __IMPORT_DESCRIPTOR_api-ms-win-crt-heap-l1-1-0 000000018000840c     ucrt:api-ms-win-crt-heap-l1-1-0.dll
 0002:00003420       __IMPORT_DESCRIPTOR_api-ms-win-crt-runtime-l1-1-0 0000000180008420     ucrt:api-ms-win-crt-runtime-l1-1-0.dll
 0002:00003434       __IMPORT_DESCRIPTOR_api-ms-win-crt-convert-l1-1-0 0000000180008434     ucrt:api-ms-win-crt-convert-l1-1-0.dll
 0002:00003448       __IMPORT_DESCRIPTOR_api-ms-win-crt-stdio-l1-1-0 0000000180008448     ucrt:api-ms-win-crt-stdio-l1-1-0.dll
 0002:0000345c       __IMPORT_DESCRIPTOR_api-ms-win-crt-string-l1-1-0 000000018000845c     ucrt:api-ms-win-crt-string-l1-1-0.dll
 0002:00003470       __NULL_IMPORT_DESCRIPTOR   0000000180008470     kernel32:KERNEL32.dll
 0003:00000030       _Init_global_epoch         0000000180009030     MSVCRT:thread_safe_statics.obj
 0003:00000040       __security_cookie          0000000180009040     MSVCRT:gs_cookie.obj
 0003:00000048       __security_cookie_complement 0000000180009048     MSVCRT:gs_cookie.obj
 0003:00000050       __scrt_native_dllmain_reason 0000000180009050     MSVCRT:utility.obj
 0003:00000058       __isa_available            0000000180009058     MSVCRT:cpu_disp.obj
 0003:0000005c       __isa_enabled              000000018000905c     MSVCRT:cpu_disp.obj
 0003:00000060       __memset_fast_string_threshold 0000000180009060     MSVCRT:cpu_disp.obj
 0003:00000068       __memset_nt_threshold      0000000180009068     MSVCRT:cpu_disp.obj
 0003:00000070       __scrt_ucrt_dll_is_in_use  0000000180009070     MSVCRT:ucrt_stubs.obj
 0003:00000080       g_wrongHeapCallbacks       0000000180009080     libextevents001.obj
 0003:00000100       g_szTagInfo                0000000180009100     libextevents001.obj
 0003:00002040       g_tagFlags                 000000018000b040     libextevents001.obj
 0003:00002428       g_refsToVerifyCnt          000000018000b428     libextevents001.obj
 0003:0000242c       g_fakeUserData             000000018000b42c     libextevents001.obj
 0003:00002430       g_tagVisitCount            000000018000b430     libextevents001.obj
 0003:000033d0       g_refsToVerify             000000018000c3d0     libextevents001.obj
 0003:0001aad0       g_userDataError            0000000180023ad0     libextevents001.obj
 0003:0001ac70       ?_OptionsStorage@?1??__local_stdio_printf_options@@9@4_KA 0000000180023c70     libextevents001.obj
 0003:0001b238       _tls_index                 0000000180024238     MSVCRT:tlssup.obj
 0003:0001b240       __scrt_current_native_startup_state 0000000180024240     MSVCRT:utility.obj
 0003:0001b248       __scrt_native_startup_lock 0000000180024248     MSVCRT:utility.obj
 0003:0001b288       __scrt_debugger_hook_flag  0000000180024288     MSVCRT:utility_desktop.obj
 0003:0001b290       ?__type_info_root_node@@3U__type_info_node@@A 0000000180024290     MSVCRT:tncleanup.obj
 0003:0001b2a0       ?_OptionsStorage@?1??__local_stdio_scanf_options@@9@4_KA 00000001800242a0     MSVCRT:default_local_stdio_options.obj
 0003:0001b2a8       __favor                    00000001800242a8     MSVCRT:cpu_disp.obj
 0003:0001b2b0       __dyn_tls_init_callback    00000001800242b0     <common>

 entry point at        0001:00003190

 Static symbols

 0000:fffd9000       .debug$S                   0000000180000000     extevents001.exp
 0000:fffd9000       .debug$S                   0000000180000000     vcruntime:VCRUNTIME140.dll
 0000:fffd9000       .debug$S                   0000000180000000     vcruntime:VCRUNTIME140.dll
 0000:fffd9000       .debug$S                   0000000180000000     vcruntime:VCRUNTIME140.dll
 0000:fffd9000       .debug$S                   0000000180000000     vcruntime:VCRUNTIME140.dll
 0000:fffd9000       .debug$S                   0000000180000000     vcruntime:VCRUNTIME140.dll
 0000:fffd9000       .debug$S                   0000000180000000     vcruntime:VCRUNTIME140.dll
 0000:fffd9000       .debug$S                   0000000180000000     vcruntime:VCRUNTIME140.dll
 0000:fffd9000       .debug$S                   0000000180000000     vcruntime:VCRUNTIME140.dll
 0000:fffd9000       .debug$S                   0000000180000000     ucrt:api-ms-win-crt-convert-l1-1-0.dll
 0000:fffd9000       .debug$S                   0000000180000000     ucrt:api-ms-win-crt-heap-l1-1-0.dll
 0000:fffd9000       .debug$S                   0000000180000000     ucrt:api-ms-win-crt-heap-l1-1-0.dll
 0000:fffd9000       .debug$S                   0000000180000000     ucrt:api-ms-win-crt-heap-l1-1-0.dll
 0000:fffd9000       .debug$S                   0000000180000000     ucrt:api-ms-win-crt-heap-l1-1-0.dll
 0000:fffd9000       .debug$S                   0000000180000000     ucrt:api-ms-win-crt-runtime-l1-1-0.dll
 0000:fffd9000       .debug$S                   0000000180000000     ucrt:api-ms-win-crt-runtime-l1-1-0.dll
 0000:fffd9000       .debug$S                   0000000180000000     ucrt:api-ms-win-crt-runtime-l1-1-0.dll
 0000:fffd9000       .debug$S                   0000000180000000     ucrt:api-ms-win-crt-runtime-l1-1-0.dll
 0000:fffd9000       .debug$S                   0000000180000000     ucrt:api-ms-win-crt-runtime-l1-1-0.dll
 0000:fffd9000       .debug$S                   0000000180000000     ucrt:api-ms-win-crt-runtime-l1-1-0.dll
 0000:fffd9000       .debug$S                   0000000180000000     ucrt:api-ms-win-crt-runtime-l1-1-0.dll
 0000:fffd9000       .debug$S                   0000000180000000     ucrt:api-ms-win-crt-runtime-l1-1-0.dll
 0000:fffd9000       .debug$S                   0000000180000000     ucrt:api-ms-win-crt-runtime-l1-1-0.dll
 0000:fffd9000       .debug$S                   0000000180000000     ucrt:api-ms-win-crt-runtime-l1-1-0.dll
 0000:fffd9000       .debug$S                   0000000180000000     ucrt:api-ms-win-crt-runtime-l1-1-0.dll
 0000:fffd9000       .debug$S                   0000000180000000     ucrt:api-ms-win-crt-runtime-l1-1-0.dll
 0000:fffd9000       .debug$S                   0000000180000000     ucrt:api-ms-win-crt-runtime-l1-1-0.dll
 0000:fffd9000       .debug$S                   0000000180000000     ucrt:api-ms-win-crt-runtime-l1-1-0.dll
 0000:fffd9000       .debug$S                   0000000180000000     ucrt:api-ms-win-crt-runtime-l1-1-0.dll
 0000:fffd9000       .debug$S                   0000000180000000     ucrt:api-ms-win-crt-runtime-l1-1-0.dll
 0000:fffd9000       .debug$S                   0000000180000000     ucrt:api-ms-win-crt-stdio-l1-1-0.dll
 0000:fffd9000       .debug$S                   0000000180000000     ucrt:api-ms-win-crt-stdio-l1-1-0.dll
 0000:fffd9000       .debug$S                   0000000180000000     ucrt:api-ms-win-crt-stdio-l1-1-0.dll
 0000:fffd9000       .debug$S                   0000000180000000     ucrt:api-ms-win-crt-stdio-l1-1-0.dll
 0000:fffd9000       .debug$S                   0000000180000000     ucrt:api-ms-win-crt-stdio-l1-1-0.dll
 0000:fffd9000       .debug$S                   0000000180000000     ucrt:api-ms-win-crt-stdio-l1-1-0.dll
 0000:fffd9000       .debug$S                   0000000180000000     ucrt:api-ms-win-crt-stdio-l1-1-0.dll
 0000:fffd9000       .debug$S                   0000000180000000     ucrt:api-ms-win-crt-stdio-l1-1-0.dll
 0000:fffd9000       .debug$S                   0000000180000000     ucrt:api-ms-win-crt-stdio-l1-1-0.dll
 0000:fffd9000       .debug$S                   0000000180000000     ucrt:api-ms-win-crt-stdio-l1-1-0.dll
 0000:fffd9000       .debug$S                   0000000180000000     ucrt:api-ms-win-crt-string-l1-1-0.dll
 0000:fffd9000       .debug$S                   0000000180000000     ucrt:api-ms-win-crt-string-l1-1-0.dll
 0000:fffd9000       .debug$S                   0000000180000000     ucrt:api-ms-win-crt-string-l1-1-0.dll
 0000:fffd9000       .debug$S                   0000000180000000     ucrt:api-ms-win-crt-string-l1-1-0.dll
 0000:fffd9000       .debug$S                   0000000180000000     ucrt:api-ms-win-crt-string-l1-1-0.dll
 0000:fffd9000       .debug$S                   0000000180000000     ucrt:api-ms-win-crt-string-l1-1-0.dll
 0000:fffd9000       .debug$S                   0000000180000000     ucrt:api-ms-win-crt-string-l1-1-0.dll
 0000:fffd9000       .debug$S                   0000000180000000     ucrt:api-ms-win-crt-string-l1-1-0.dll
 0000:fffd9000       .debug$S                   0000000180000000     kernel32:KERNEL32.dll
 0000:fffd9000       .debug$S                   0000000180000000     kernel32:KERNEL32.dll
 0000:fffd9000       .debug$S                   0000000180000000     kernel32:KERNEL32.dll
 0000:fffd9000       .debug$S                   0000000180000000     kernel32:KERNEL32.dll
 0000:fffd9000       .debug$S                   0000000180000000     kernel32:KERNEL32.dll
 0000:fffd9000       .debug$S                   0000000180000000     kernel32:KERNEL32.dll
 0000:fffd9000       .debug$S                   0000000180000000     kernel32:KERNEL32.dll
 0000:fffd9000       .debug$S                   0000000180000000     kernel32:KERNEL32.dll
 0000:fffd9000       .debug$S                   0000000180000000     kernel32:KERNEL32.dll
 0000:fffd9000       .debug$S                   0000000180000000     kernel32:KERNEL32.dll
 0000:fffd9000       .debug$S                   0000000180000000     kernel32:KERNEL32.dll
 0000:fffd9000       .debug$S                   0000000180000000     kernel32:KERNEL32.dll
 0000:fffd9000       .debug$S                   0000000180000000     kernel32:KERNEL32.dll
 0000:fffd9000       .debug$S                   0000000180000000     kernel32:KERNEL32.dll
 0000:fffd9000       .debug$S                   0000000180000000     kernel32:KERNEL32.dll
 0000:fffd9000       .debug$S                   0000000180000000     kernel32:KERNEL32.dll
 0000:fffd9000       .debug$S                   0000000180000000     kernel32:KERNEL32.dll
 0000:fffd9000       .debug$S                   0000000180000000     kernel32:KERNEL32.dll
 0000:fffd9000       .debug$S                   0000000180000000     kernel32:KERNEL32.dll
 0000:fffd9000       .debug$S                   0000000180000000     kernel32:KERNEL32.dll
 0000:fffd9000       .debug$S                   0000000180000000     kernel32:KERNEL32.dll
 0000:fffd9000       .debug$S                   0000000180000000     kernel32:KERNEL32.dll
 0000:fffd9000       .debug$S                   0000000180000000     kernel32:KERNEL32.dll
 0000:fffd9000       .debug$S                   0000000180000000     kernel32:KERNEL32.dll
 0000:fffd9000       .debug$S                   0000000180000000     kernel32:KERNEL32.dll
 0000:fffd9000       .debug$S                   0000000180000000     kernel32:KERNEL32.dll
 0000:fffd9000       .debug$S                   0000000180000000     kernel32:KERNEL32.dll
 0000:fffd9000       .debug$S                   0000000180000000     kernel32:KERNEL32.dll
 0001:00000e00       addRefToVerify             0000000180001e00 f   libextevents001.obj
 0001:00000e6c       agentProc                  0000000180001e6c f   libextevents001.obj
 0001:00000fa0       agentThreadWrapper         0000000180001fa0 f   libextevents001.obj
 0001:0000110c       checkExtensions            000000018000210c f   libextevents001.obj
 0001:0000186c       check_option               000000018000286c f   libextevents001.obj
 0001:00001ab4       file_basename              0000000180002ab4 f   libextevents001.obj
 0001:00002678       startAgentThreadWrapper    0000000180003678 f   libextevents001.obj
 0001:000029b8       syncDebuggeeStatus         00000001800039b8 f   libextevents001.obj
 0001:00002c58       capture_previous_context   0000000180003c58 f   MSVCRT:gs_report.obj
 0001:00002ccc       ?__scrt_initialize_thread_safe_statics@@YAHXZ 0000000180003ccc f   MSVCRT:thread_safe_statics.obj
 0001:00002d9c       ?__scrt_uninitialize_thread_safe_statics@@YAXXZ 0000000180003d9c f   MSVCRT:thread_safe_statics.obj
 0001:00002e40       $$000000                   0000000180003e40     MSVCRT:amdsecgs.obj
 0001:00002e70       ?dllmain_crt_dispatch@@YAHQEAUHINSTANCE__@@KQEAX@Z 0000000180003e70 f   MSVCRT:dll_dllmain.obj
 0001:00002ec0       ?dllmain_crt_process_attach@@YAHQEAUHINSTANCE__@@QEAX@Z 0000000180003ec0 f   MSVCRT:dll_dllmain.obj
 0001:00002fd8       ?dllmain_crt_process_detach@@YAH_N@Z 0000000180003fd8 f   MSVCRT:dll_dllmain.obj
 0001:0000305c       ?dllmain_dispatch@@YAHQEAUHINSTANCE__@@KQEAX@Z 000000018000405c f   MSVCRT:dll_dllmain.obj
 0001:00003a80       $$000000                   0000000180004a80     MSVCRT:guard_dispatch.obj
 0001:00003aa0       $$000000                   0000000180004aa0     MSVCRT:guard_xfg_dispatch.obj
 0001:00003ab6       ?fin$0@?0??dllmain_crt_process_attach@@YAHQEAUHINSTANCE__@@QEAX@Z@4HA 0000000180004ab6 f   MSVCRT:dll_dllmain.obj
 0001:00003acd       ?fin$0@?0??dllmain_crt_process_detach@@YAH_N@Z@4HA 0000000180004acd f   MSVCRT:dll_dllmain.obj
 0001:00003ae6       ?fin$1@?0??dllmain_crt_process_detach@@YAH_N@Z@4HA 0000000180004ae6 f   MSVCRT:dll_dllmain.obj
 0001:00003afa       ?filt$0@?0??dllmain_dispatch@@YAHQEAUHINSTANCE__@@KQEAX@Z@4HA 0000000180004afa f   MSVCRT:dll_dllmain.obj
 0001:00003b30       __scrt_is_nonwritable_in_current_image$filt$0 0000000180004b30 f   MSVCRT:utility.obj
 0002:00000220       ?__scrt_initialize_tss_var@@3P6AHXZEA 0000000180005220     MSVCRT:thread_safe_statics.obj
 0002:00000340       ?opcLengths@@3QBEB         0000000180005340     libextevents001.obj
 0002:00002610       GS_ExceptionPointers       0000000180007610     MSVCRT:gs_report.obj
 0002:00002d30       $unwind$fprintf            0000000180007d30     libextevents001.obj
 0002:00002d3c       $unwind$printf             0000000180007d3c     libextevents001.obj
 0002:00002d48       $unwind$?NewObject@JNIEnv_@@QEAAPEAV_jobject@@PEAV_jclass@@PEAU_jmethodID@@ZZ 0000000180007d48     libextevents001.obj
 0002:00002d48       $unwind$nsk_lcomplain      0000000180007d48     libextevents001.obj
 0002:00002d48       $unwind$nsk_ldisplay       0000000180007d48     libextevents001.obj
 0002:00002d50       $unwind$nsk_jvmti_waitForSync 0000000180007d50     libextevents001.obj
 0002:00002d50       $unwind$nsk_lvdisplay      0000000180007d50     libextevents001.obj
 0002:00002d50       $unwind$_RTC_Initialize    0000000180007d50     MSVCRT:initsect.obj
 0002:00002d50       $unwind$_RTC_Terminate     0000000180007d50     MSVCRT:initsect.obj
 0002:00002d50       $unwind$?__scrt_initialize_thread_safe_statics@@YAHXZ 0000000180007d50     MSVCRT:thread_safe_statics.obj
 0002:00002d5c       $unwind$nsk_complain       0000000180007d5c     libextevents001.obj
 0002:00002d5c       $unwind$nsk_printf         0000000180007d5c     libextevents001.obj
 0002:00002d64       $unwind$nsk_lvcomplain     0000000180007d64     libextevents001.obj
 0002:00002d7c       $unwind$nsk_ltrace         0000000180007d7c     libextevents001.obj
 0002:00002d7c       $unwind$__report_gsfailure 0000000180007d7c     MSVCRT:gs_report.obj
 0002:00002d84       $unwind$nsk_lvtrace        0000000180007d84     libextevents001.obj
 0002:00002d84       $unwind$__raise_securityfailure 0000000180007d84     MSVCRT:gs_report.obj
 0002:00002d84       $unwind$__scrt_initialize_crt 0000000180007d84     MSVCRT:utility.obj
 0002:00002d84       $unwind$__scrt_initialize_onexit_tables 0000000180007d84     MSVCRT:utility.obj
 0002:00002d84       $unwind$__scrt_release_startup_lock 0000000180007d84     MSVCRT:utility.obj
 0002:00002d84       $unwind$__scrt_uninitialize_crt 0000000180007d84     MSVCRT:utility.obj
 0002:00002d84       $unwind$_onexit            0000000180007d84     MSVCRT:utility.obj
 0002:00002d8c       $unwind$nsk_lverify        0000000180007d8c     libextevents001.obj
 0002:00002d9c       $unwind$nsk_vprintf        0000000180007d9c     libextevents001.obj
 0002:00002dac       $unwind$?nsk_jni_lverify@@YAHHPEAUJNIEnv_@@HQEBDH1ZZ 0000000180007dac     libextevents001.obj
 0002:00002dc0       $unwind$?nsk_jni_check_exception@@YAHPEAUJNIEnv_@@QEBDH@Z 0000000180007dc0     libextevents001.obj
 0002:00002ddc       $unwind$nsk_jvmti_parseOptions 0000000180007ddc     libextevents001.obj
 0002:00002df8       $unwind$nsk_jvmti_createJVMTIEnv 0000000180007df8     libextevents001.obj
 0002:00002e0c       $unwind$Java_nsk_jvmti_unit_FollowReferences_FollowRefObjects_resetTags 0000000180007e0c     libextevents001.obj
 0002:00002e0c       $unwind$addRefToVerify     0000000180007e0c     libextevents001.obj
 0002:00002e0c       $unwind$nsk_jvmti_resetAgentData 0000000180007e0c     libextevents001.obj
 0002:00002e0c       $unwind$nsk_jvmti_resumeSync 0000000180007e0c     libextevents001.obj
 0002:00002e0c       $unwind$nsk_jvmti_setFailStatus 0000000180007e0c     libextevents001.obj
 0002:00002e0c       $unwind$__scrt_initialize_default_local_stdio_options 0000000180007e0c     MSVCRT:default_local_stdio_options.obj
 0002:00002e0c       $unwind$?dllmain_crt_dispatch@@YAHQEAUHINSTANCE__@@KQEAX@Z 0000000180007e0c     MSVCRT:dll_dllmain.obj
 0002:00002e0c       $unwind$DllMain            0000000180007e0c     MSVCRT:dll_dllmain_stub.obj
 0002:00002e0c       $unwind$__GSHandlerCheck   0000000180007e0c     MSVCRT:gshandler.obj
 0002:00002e0c       $unwind$?__scrt_uninitialize_thread_safe_statics@@YAXXZ 0000000180007e0c     MSVCRT:thread_safe_statics.obj
 0002:00002e0c       $unwind$__scrt_acquire_startup_lock 0000000180007e0c     MSVCRT:utility.obj
 0002:00002e0c       $unwind$__scrt_dllmain_after_initialize_c 0000000180007e0c     MSVCRT:utility.obj
 0002:00002e0c       $unwind$__scrt_dllmain_before_initialize_c 0000000180007e0c     MSVCRT:utility.obj
 0002:00002e0c       $unwind$__scrt_dllmain_crt_thread_attach 0000000180007e0c     MSVCRT:utility.obj
 0002:00002e0c       $unwind$__scrt_dllmain_crt_thread_detach 0000000180007e0c     MSVCRT:utility.obj
 0002:00002e0c       $unwind$__scrt_dllmain_uninitialize_c 0000000180007e0c     MSVCRT:utility.obj
 0002:00002e0c       $unwind$__scrt_dllmain_uninitialize_critical 0000000180007e0c     MSVCRT:utility.obj
 0002:00002e0c       $unwind$atexit             0000000180007e0c     MSVCRT:utility.obj
 0002:00002e14       $unwind$nsk_jvmti_lverify  0000000180007e14     libextevents001.obj
 0002:00002e28       $unwind$exitOnError        0000000180007e28     libextevents001.obj
 0002:00002e38       $unwind$check_option       0000000180007e38     libextevents001.obj
 0002:00002e38       $unwind$_DllMainCRTStartup 0000000180007e38     MSVCRT:dll_dllmain.obj
 0002:00002e48       $unwind$Java_nsk_share_jvmti_ArgumentHandler_getAgentOptionsString 0000000180007e48     libextevents001.obj
 0002:00002e5c       $unwind$Java_nsk_jvmti_unit_FollowReferences_FollowRefObjects_getTag 0000000180007e5c     libextevents001.obj
 0002:00002e5c       $unwind$Java_nsk_share_jvmti_DebugeeClass_checkStatus 0000000180007e5c     libextevents001.obj
 0002:00002e5c       $unwind$agentThreadWrapper 0000000180007e5c     libextevents001.obj
 0002:00002e6c       $unwind$startAgentThreadWrapper 0000000180007e6c     libextevents001.obj
 0002:00002e88       $unwind$syncDebuggeeStatus 0000000180007e88     libextevents001.obj
 0002:00002e88       $unwind$__scrt_dllmain_exception_filter 0000000180007e88     MSVCRT:utility.obj
 0002:00002e9c       $unwind$Java_nsk_share_jvmti_DebugeeClass_resetAgentData 0000000180007e9c     libextevents001.obj
 0002:00002ea4       $unwind$MA_checkStatus     0000000180007ea4     libextevents001.obj
 0002:00002eb8       $unwind$Java_nsk_jvmti_unit_FollowReferences_FollowRefObjects_setTag 0000000180007eb8     libextevents001.obj
 0002:00002ed0       $unwind$Java_nsk_jvmti_unit_FollowReferences_FollowRefObjects_addRefToVerify 0000000180007ed0     libextevents001.obj
 0002:00002eec       $unwind$Agent_Initialize   0000000180007eec     libextevents001.obj
 0002:00002f04       $unwind$checkExtensions    0000000180007f04     libextevents001.obj
 0002:00002f1c       $unwind$agentProc          0000000180007f1c     libextevents001.obj
 0002:00002f34       $unwind$capture_previous_context 0000000180007f34     MSVCRT:gs_report.obj
 0002:00002f40       $unwind$__GSHandlerCheckCommon 0000000180007f40     MSVCRT:gshandler.obj
 0002:00002f48       $xdatasym                  0000000180007f48     MSVCRT:amdsecgs.obj
 0002:00002f4c       $unwind$?dllmain_crt_process_attach@@YAHQEAUHINSTANCE__@@QEAX@Z 0000000180007f4c     MSVCRT:dll_dllmain.obj
 0002:00002f88       $unwind$?fin$0@?0??dllmain_crt_process_attach@@YAHQEAUHINSTANCE__@@QEAX@Z@4HA 0000000180007f88     MSVCRT:dll_dllmain.obj
 0002:00002f88       $unwind$?fin$0@?0??dllmain_crt_process_detach@@YAH_N@Z@4HA 0000000180007f88     MSVCRT:dll_dllmain.obj
 0002:00002f88       $unwind$?fin$1@?0??dllmain_crt_process_detach@@YAH_N@Z@4HA 0000000180007f88     MSVCRT:dll_dllmain.obj
 0002:00002f90       $unwind$?dllmain_crt_process_detach@@YAH_N@Z 0000000180007f90     MSVCRT:dll_dllmain.obj
 0002:00002fe4       $unwind$?dllmain_dispatch@@YAHQEAUHINSTANCE__@@KQEAX@Z 0000000180007fe4     MSVCRT:dll_dllmain.obj
 0002:0000300c       $unwind$?filt$0@?0??dllmain_dispatch@@YAHQEAUHINSTANCE__@@KQEAX@Z@4HA 000000018000800c     MSVCRT:dll_dllmain.obj
 0002:00003014       $unwind$__scrt_is_nonwritable_in_current_image 0000000180008014     MSVCRT:utility.obj
 0002:00003034       $unwind$__scrt_is_nonwritable_in_current_image$filt$0 0000000180008034     MSVCRT:utility.obj
 0002:0000303c       $unwind$__scrt_fastfail    000000018000803c     MSVCRT:utility_desktop.obj
 0002:0000304c       $unwind$__security_init_cookie 000000018000804c     MSVCRT:gs_support.obj
 0002:00003058       $unwind$__isa_available_init 0000000180008058     MSVCRT:cpu_disp.obj
 0002:00003068       $xdatasym                  0000000180008068     MSVCRT:guard_dispatch.obj
 0002:00003070       $xdatasym                  0000000180008070     MSVCRT:guard_xfg_dispatch.obj
 0002:00003080       .edata                     0000000180008080     extevents001.exp
 0002:000030a8       rgpv                       00000001800080a8     extevents001.exp
 0002:000030e0       rgszName                   00000001800080e0     extevents001.exp
 0002:00003118       rgwOrd                     0000000180008118     extevents001.exp
 0002:00003134       szName                     0000000180008134     extevents001.exp
 0002:00003145       $N00001                    0000000180008145     extevents001.exp
 0002:00003154       $N00002                    0000000180008154     extevents001.exp
 0002:00003161       $N00003                    0000000180008161     extevents001.exp
 0002:000031a6       $N00004                    00000001800081a6     extevents001.exp
 0002:000031e3       $N00005                    00000001800081e3     extevents001.exp
 0002:0000322b       $N00006                    000000018000822b     extevents001.exp
 0002:0000326b       $N00007                    000000018000826b     extevents001.exp
 0002:000032a8       $N00008                    00000001800082a8     extevents001.exp
 0002:000032e3       $N00009                    00000001800082e3     extevents001.exp
 0002:00003311       $N00010                    0000000180008311     extevents001.exp
 0002:00003342       $N00011                    0000000180008342     extevents001.exp
 0002:00003371       $N00012                    0000000180008371     extevents001.exp
 0002:000033a0       $N00013                    00000001800083a0     extevents001.exp
 0002:000033d5       $N00014                    00000001800083d5     extevents001.exp
 0002:00003842       .idata$6                   0000000180008842     kernel32:KERNEL32.dll
 0002:000038b0       .idata$6                   00000001800088b0     vcruntime:VCRUNTIME140.dll
 0002:00003a42       .idata$6                   0000000180008a42     ucrt:api-ms-win-crt-heap-l1-1-0.dll
 0002:00003a62       .idata$6                   0000000180008a62     ucrt:api-ms-win-crt-runtime-l1-1-0.dll
 0002:00003a84       .idata$6                   0000000180008a84     ucrt:api-ms-win-crt-convert-l1-1-0.dll
 0002:00003aa6       .idata$6                   0000000180008aa6     ucrt:api-ms-win-crt-stdio-l1-1-0.dll
 0002:00003ac6       .idata$6                   0000000180008ac6     ucrt:api-ms-win-crt-string-l1-1-0.dll
 0003:00000000       ?codeAttributeName@@3PEBDEB 0000000180009000     libextevents001.obj
 0003:00000008       ?lineNumberAttributeName@@3PEBDEB 0000000180009008     libextevents001.obj
 0003:00000010       ?localVarAttributeName@@3PEBDEB 0000000180009010     libextevents001.obj
 0003:00000018       ?localVarTypeAttributeName@@3PEBDEB 0000000180009018     libextevents001.obj
 0003:00000020       ?stackMapAttributeName@@3PEBDEB 0000000180009020     libextevents001.obj
 0003:00000028       ?callBytes@@3PAEA          0000000180009028     libextevents001.obj
 0003:0000002c       ?allocBytes@@3PAEA         000000018000902c     libextevents001.obj
 0003:0001aad4       redefineAttempted          0000000180023ad4     libextevents001.obj
 0003:0001aad8       nsk_context                0000000180023ad8     libextevents001.obj
 0003:0001aae4       redefineSucceed            0000000180023ae4     libextevents001.obj
 0003:0001aae8       agentFailed                0000000180023ae8     libextevents001.obj
 0003:0001aaec       currentAgentStatus         0000000180023aec     libextevents001.obj
 0003:0001aaf0       context                    0000000180023af0     libextevents001.obj
 0003:0001aba8       agentThread                0000000180023ba8     libextevents001.obj
 0003:0001abb0       agentThreadProc            0000000180023bb0     libextevents001.obj
 0003:0001abb8       agentThreadArg             0000000180023bb8     libextevents001.obj
 0003:0001abc0       agent_data                 0000000180023bc0     libextevents001.obj
 0003:0001abd0       jvmti_env                  0000000180023bd0     libextevents001.obj
 0003:0001abd8       jvm                        0000000180023bd8     libextevents001.obj
 0003:0001abe0       jni_env                    0000000180023be0     libextevents001.obj
 0003:0001abe8       checkStatus_func           0000000180023be8     libextevents001.obj
 0003:0001abf0       ?codeAttributeIndex@@3GA   0000000180023bf0     libextevents001.obj
 0003:0001abf4       ?lineNumberAttributeIndex@@3GA 0000000180023bf4     libextevents001.obj
 0003:0001abf8       ?localVarAttributeIndex@@3GA 0000000180023bf8     libextevents001.obj
 0003:0001abfc       ?localVarTypeAttributeIndex@@3GA 0000000180023bfc     libextevents001.obj
 0003:0001ac00       ?stackMapAttributeIndex@@3GA 0000000180023c00     libextevents001.obj
 0003:0001ac04       ?stackFrameOffset@@3GA     0000000180023c04     libextevents001.obj
 0003:0001ac08       ?mode@@3HA                 0000000180023c08     libextevents001.obj
 0003:0001ac0c       ?constantPoolSize@@3GA     0000000180023c0c     libextevents001.obj
 0003:0001ac10       ?orig@@3PEBEEB             0000000180023c10     libextevents001.obj
 0003:0001ac18       ?gen@@3PEAEEA              0000000180023c18     libextevents001.obj
 0003:0001ac20       ?inputPos@@3PEAEEA         0000000180023c20     libextevents001.obj
 0003:0001ac28       ?endPos@@3PEBEEB           0000000180023c28     libextevents001.obj
 0003:0001ac30       ?genPos@@3PEAEEA           0000000180023c30     libextevents001.obj
 0003:0001ac38       ?markPos@@3PEAEEA          0000000180023c38     libextevents001.obj
 0003:0001ac40       ?constantPool@@3PEAPEADEA  0000000180023c40     libextevents001.obj
 0003:0001ac48       ?constantPoolCount@@3GA    0000000180023c48     libextevents001.obj
 0003:0001ac4c       ?zeroBytes@@3PAEA          0000000180023c4c     libextevents001.obj
 0003:0001ac50       ?codeLength@@3IA           0000000180023c50     libextevents001.obj
 0003:0001ac58       ?map@@3PEAIEA              0000000180023c58     libextevents001.obj
 0003:0001ac60       ?widening@@3PEACEA         0000000180023c60     libextevents001.obj
 0003:0001ac68       timeout                    0000000180023c68     libextevents001.obj
 0003:0001ac80       GS_ExceptionRecord         0000000180023c80     MSVCRT:gs_report.obj
 0003:0001ad20       GS_ContextRecord           0000000180023d20     MSVCRT:gs_report.obj
 0003:0001b1f0       ?g_tss_cv@@3U_RTL_CONDITION_VARIABLE@@A 00000001800241f0     MSVCRT:thread_safe_statics.obj
 0003:0001b1f8       ?g_tss_event@@3PEAXEA      00000001800241f8     MSVCRT:thread_safe_statics.obj
 0003:0001b200       ?g_tss_mutex@@3U_RTL_CRITICAL_SECTION@@A 0000000180024200     MSVCRT:thread_safe_statics.obj
 0003:0001b228       ?g_sleep_condition_variable_cs@@3P6AHPEAU_RTL_CONDITION_VARIABLE@@PEAU_RTL_CRITICAL_SECTION@@K@ZEA 0000000180024228     MSVCRT:thread_safe_statics.obj
 0003:0001b230       ?g_wake_all_condition_variable@@3P6AXPEAU_RTL_CONDITION_VARIABLE@@@ZEA 0000000180024230     MSVCRT:thread_safe_statics.obj
 0003:0001b23c       ?__proc_attached@@3HA      000000018002423c     MSVCRT:dll_dllmain.obj
 0003:0001b250       ?is_initialized_as_dll@@3_NA 0000000180024250     MSVCRT:utility.obj
 0003:0001b251       ?module_local_atexit_table_initialized@@3_NA 0000000180024251     MSVCRT:utility.obj
 0003:0001b258       ?module_local_atexit_table@@3U_onexit_table_t@@A 0000000180024258     MSVCRT:utility.obj
 0003:0001b270       ?module_local_at_quick_exit_table@@3U_onexit_table_t@@A 0000000180024270     MSVCRT:utility.obj
